:020000040000FA
:08000800B529A501A601A7011D
:10001000A801A901AA01AB01AC01AD01AE01AF017C
:10002000B001B5010800850107309F00831600303C
:1000300085004030860083128501860106309000DD
:100040001010080028305820051003304A20552091
:10005000851485105020851485105020051002301D
:100060004A205020283042201030422001304220C7
:1000700055200800A300230E05144A202308051468
:100080004A200800A300230E05104A20230805106B
:100090004A2008000F39860085148510502008007A
:1000A0002930FF3E031D5128080005305828FA303A
:1000B000A400FE3051200000A40B59280800643031
:1000C000B200B20B61280800803042200C30422080
:1000D000080020303A2020303A2020303A202030CA
:1000E0003A2020303A2020303A2020303A20203068
:1000F0003A20C03042200C30422008002508303E13
:100100003A202608303E3A202708303E3A202E304A
:100110003A202808303E3A202908303E3A20203044
:100120003A206B303A2048303A207A303A200800A2
:100130002508303E3A202608303E3A202708303E37
:100140003A202808303E3A202908303E3A20203014
:100150003A2020303A2048303A207A303A20203075
:100160003A2008002508303E3A202E303A20260852
:10017000303E3A202708303E3A202808303E3A20C8
:100180002908303E3A2020303A204D303A2048307D
:100190003A207A303A2008002508303E3A202608D6
:1001A000303E3A202E303A202708303E3A202808A8
:1001B000303E3A202908303E3A2020303A204D3057
:1001C0003A2048303A207A303A20080046303A2027
:1001D00072303A2071303A203A303A2020303A20BA
:1001E00008002A082A0E0F39F03EAE00AE07E23EA4
:1001F000B000323EAD002A080F39B007B007AD0796
:10020000E93EAC00AC07AC072B0E0F39AC07AD07CD
:10021000AC0DAD0DAD09AD0D2B080F39AD07AE0D11
:100220000730AF000A30AD07AC03031C1329AC073D
:10023000B003031C1729B007AE03031C1B29AE072C
:10024000AF03031C1F2900343708AA003608AB008F
:10025000F1202F08A5002E08A6003008A7002C08C2
:10026000A8002D08A9000800B601B7010A30A000B7
:10027000B030B1008F018E010C101014BD30B200EF
:10028000B20B4029B10B3E29AF30B100A00B3E2983
:100290003230B300B30B4A2910100F08B7000E0814
:1002A000B600B5010800B601B701AE30B1008F014C
:1002B0008E010C101014BE30B200B20B5D29B10BD0
:1002C0005B292930B300B30B632910100F08B70066
:1002D0000E08B6000130B5000800B601B70156306F
:1002E000B1008F018E010C1010142430B200B20B3B
:1002F0007729B10B75297A30B300B30B7D29000043
:1003000010100F08B7000E08B6000230B500080044
:1003100016309000B601B7010C108F018E01101439
:10032000FA30B300B30B9229FA30B300B30B96291D
:10033000A430B300B30B9A290000000000000000B5
:1003400010100F08B7000E08B600063090000330FA
:10035000B50008003230B100861206165F208616FE
:1003600006125F20B10BAC290800052013202220C3
:10037000AA2134210C1853210C186D210C18882146
:1003800024216420E620003035060319982001302E
:10039000350603197E20023035060319B2200330DA
:0803A00035060319CC20B92930
:02400E00023F6F
:00000001FF
